:100000008A110A120528000009000730990083169A
:10001000051085100511851285150512831205102E
:1000200085100511851105128512AE010130AE0053
:1000300005162E08013C031D3428AE01AC012C0826
:10004000C83C031C3128851D27280130AE001F3015
:1000500083050A30A000A101F4210130AC07031C84
:100060001F281F30830519281F308305AE01051294
:100070009420AC012C08193C031C5228AD012D081A
:100080003B3C031C4C28E830A0000330A100F421C5
:100090000130AD07031C3F281F3083050130AC073A
:1000A000031C3A281F3083050130AE0005162E08C8
:1000B000013C031D7228AE01AC012C08C83C031C96
:1000C0006F28851D65280130AE001F3083050A307A
:1000D000A000A101F4210130AC07031C5D281F30F2
:1000E000830557281F308305AE010512AC20AC01F3
:1000F0002C08193C031C9028AD012D083B3C031C27
:100100008A28E830A0000330A100F4210130AD07B7
:10011000031C7D281F3083050130AC07031C7828A1
:100120001F3083051628932805145830A00002308C
:10013000A100F421CE209C21D7209C213E219C218E
:100140000C219C211A219C21E720E830A0000330DB
:10015000A100F4210510080005148516AD012D0835
:100160000A3C031CBC28E830A0000330A100F421A5
:100170000130AD07031CAF281F308305E830A00015
:100180000330A100F421851205100800C021D121FF
:100190000800D121C021C021C0210800D121C021E7
:1001A000D121C0210800D121C021C0210800C021D7
:1001B0000800C021C021D121C0210800D121D121B6
:1001C000C0210800C021C021C021C0210800C021D9
:1001D000C0210800C021D121D121D1210800D12185
:1001E000C021D1210800C021D121C021C021080097
:1001F000D121D1210800D121C0210800D121D12154
:10020000D1210800C021D121D121C0210800D12154
:10021000D121C021D1210800C021D121C021080055
:10022000C021C021C0210800D1210800C021C02167
:10023000D1210800C021C021C021D1210800C02146
:10024000D121D1210800D121C021C021D121080014
:10025000D121C021D121D1210800D121D121C0211A
:10026000C0210800D121D121D121D121D1210800E3
:10027000C021D121D121D121D1210800C021C0210B
:10028000D121D121D1210800C021C021C021D121FB
:10029000D1210800C021C021C021C021D1210800E6
:1002A000C021C021C021C021C0210800D121C0210E
:1002B000C021C021C0210800D121D121C021C021ED
:1002C000C0210800D121D121D121C021C0210800A5
:1002D000D121D121D121D121C0210800C021D1219A
:1002E000C021D121C021D1210800D121D121C0219B
:1002F000C021D121D1210800C021C021D121D1218B
:10030000C021C0210800D121C021C021D121C0219C
:100310000800D121C021C021C021D1210800D12154
:10032000C021C021C021C021D121080005116430A5
:10033000A000A101F421080005116430A000A10172
:10034000F4216430A000A101F4216430A000A101D7
:10035000F421080005116430A000A101F4216430EB
:10036000A000A101F4216430A000A101F4216430B7
:10037000A000A101F4216430A000A101F421080033
:100380000515053084000230AA009930A000023023
:10039000A1004430A2000030A3002F2205119621B5
:1003A00008000515053084000230AA009930A0002D
:1003B0000230A1000E30A2000130A3002F2205114F
:1003C000962108000515053084000230AA009930F6
:1003D000A0000230A100EE30A2000230A3002F22C4
:1003E000051196210800F329A0080319FF29062208
:1003F000A00300000000000000000000F429A10894
:10040000031908000622A103A003F4290C30A5005B
:10041000A50B082A000000001230A200A20B152A2A
:100420001722172200000000080017220E2A0D30A4
:10043000A400A40B192A000008001030A802000133
:10044000031C013EA902031C0800262A0A30A80248
:100450000001031C013EA902031C0800262A2A08E9
:1004600080042008A8002108A9001D220130A20252
:10047000031CA3032A0980052008A8002108A9005D
:100480001D22A208031D2F2AA308031D2F2A0800DE
:02400E00C433B9
:00000001FF
